:1000000012C08CC120C01FC01EC01DC01CC01BC0A0
:1000100054C1F7C118C017C016C015C014C013C012
:1000200012C011C010C011241FBECFE5D4E0DEBF46
:10003000CDBF10E0A0E6B0E001C01D92A836B10728
:10004000E1F73DD2C0C4DCCFCF93DF93CDB7DEB7AD
:1000500087E390E02FEFFC01208388E390E0FC0130
:10006000108284E390E02FEFFC01208385E390E091
:10007000FC01108281E390E020E3FC01208382E315
:1000800090E0FC011082DF91CF910895CF93DF9330
:10009000CDB7DEB782E390E022E330E0F9012081C2
:1000A0002061FC012083DF91CF910895CF93DF93EE
:1000B000CDB7DEB782E390E022E330E0F9012081A2
:1000C0002F7EFC012083DF91CF910895CF93DF93A2
:1000D000CDB7DEB782E390E022E330E0F901208182
:1000E0002062FC012083DF91CF910895CF93DF93AD
:1000F000CDB7DEB782E390E022E330E0F901208162
:100100002F7DFC012083DF91CF910895CF93DF9362
:10011000CDB7DEB785E390E025E330E0F90120813B
:100120002062FC012083DF91CF910895CF93DF936C
:10013000CDB7DEB785E390E025E330E0F90120811B
:100140002F7DFC012083DF91CF910895CF93DF9322
:10015000CDB7DEB785E390E025E330E0F9012081FB
:100160002061FC012083DF91CF910895CF93DF932D
:10017000CDB7DEB785E390E025E330E0F9012081DB
:100180002F7EFC012083DF91CF910895CF93DF93E1
:10019000CDB7DEB785E390E025E330E0F9012081BB
:1001A0002860FC012083DF91CF910895CF93DF93E6
:1001B000CDB7DEB785E390E025E330E0F90120819B
:1001C000277FFC012083DF91CF910895CF93DF93A8
:1001D000CDB7DEB788E390E028E330E0F901208175
:1001E0002160FC012083DF91CF910895CF93DF93AD
:1001F000CDB7DEB788E390E028E330E0F901208155
:100200002E7FFC012083DF91CF910895CF93DF9360
:10021000CDB7DEB76BDF3ADFDF91CF910895CF9393
:10022000DF93CDB7DEB742DF51DFDF91CF91089585
:10023000CF93DF93CDB7DEB799DF68DFDF91CF9142
:100240000895CF93DF93CDB7DEB770DF7FDFDF9107
:10025000CF910895CF93DF93CDB7DEB7C7DF96DF99
:10026000DF91CF910895CF93DF93CDB7DEB79EDFB7
:10027000ADDFDF91CF910895CF93DF93CDB7DEB798
:1002800035DF94DF03DFA2DFDF91CF910895CF93B5
:10029000DF93CDB7DEB7AADF09DF78DF17DFDF91A5
:1002A000CF910895CF93DF93CDB7DEB7FFDE1EDF8A
:1002B0007DDF9CDFDF91CF9108951F920F92009018
:1002C0005F000F9211242F933F934F935F936F938F
:1002D0007F938F939F93AF93BF93EF93FF93CF93AE
:1002E000DF93CDB7DEB784EF91E090936100809308
:1002F00060009EDFDF91CF91FF91EF91BF91AF91B1
:100300009F918F917F916F915F914F913F912F912D
:100310000F9000925F000F901F9018951F920F9200
:1003200000905F000F9211242F938F939F93EF9370
:10033000FF93CF93DF9300D0CDB7DEB780E390E09B
:10034000FC018081882F90E084709927009779F0D4
:100350008EE490E0FC0110828CE490E0FC011182BC
:1003600010828EE490E021E0FC0120833BC080E31A
:1003700090E0FC018081882F90E08470992700979D
:1003800089F58EE490E0FC0110828CE490E0FC01A1
:10039000808191819A83898389819A818130FDE767
:1003A0009F0738F088EE93E090936100809360009F
:1003B00019C089819A8180382EE3920728F410921F
:1003C0006100109260000EC089819A8180589E431E
:1003D000929582958F7089279F70892790936100ED
:1003E000809360000F900F90DF91CF91FF91EF917C
:1003F0009F918F912F910F9000925F000F901F900F
:1004000018951F920F9200905F000F9211242F9366
:100410003F934F935F936F937F938F939F93AF938C
:10042000BF93EF93FF93CF93DF93CDB7DEB7809168
:10043000640090916500009769F4809166008823BC
:1004400011F41ADF07C080916600813011F41FDFBC
:1004500001C028DF20916400309165008091620026
:10046000909163002817390709F41CDF809164001C
:10047000909165000196909365008093640080914F
:10048000640090916500853F21E0920720F0109272
:10049000650010926400DF91CF91FF91EF91BF91C1
:1004A000AF919F918F917F916F915F914F913F910C
:1004B0002F910F9000925F000F901F901895CF938F
:1004C000DF93CDB7DEB76C970FB6F894DEBF0FBEE3
:1004D000CDBFBADD85E590E021E0FC0120838BE50E
:1004E00090E020E4FC0120838FE490E0FC01108286
:1004F00089E590E029E530E0F90120812460FC01E4
:1005000020838EE490E0FC0110828CE490E0FC01FA
:100510001182108283E590E021E0FC01208389E5CF
:1005200090E029E530E0F90120812160FC01208381
:1005300078948EE490E021E0FC012083B7DDD6DDE5
:10054000F5DD14DE33DE52DE80E090E0AAEFB3E4A6
:1005500089839A83AB83BC8320E030E04AE755E48B
:1005600069817A818B819C81A3D1DC01CB018D8350
:100570009E83AF83B88720E030E040E85FE36D8181
:100580007E818F81988513D188232CF481E090E0BF
:100590009A8789873BC020E03FEF4FE757E46D81A2
:1005A0007E818F81988580D118163CF520E030E05F
:1005B00040E251E469817A818B819C8179D1DC01AF
:1005C000CB01BC01CD01F7D0DC01CB019A87898733
:1005D0000FC080E991E09C878B878B859C85019774
:1005E000F1F79C878B8789859A8501979A878987F8
:1005F00089859A85009769F713C06D817E818F8107
:100600009885D9D0DC01CB019A87898789859A851D
:100610009E878D878D859E850197F1F79E878D87B3
:1006200007DE80E090E0A8ECB2E48F87988BA98B7E
:10063000BA8B20E030E04AE755E46F8578898989F4
:100640009A8936D1DC01CB018B8B9C8BAD8BBE8B19
:1006500020E030E040E85FE36B897C898D899E89EA
:10066000A6D088232CF481E090E0988F8F8B3BC03C
:1006700020E03FEF4FE757E46B897C898D899E89A5
:1006800013D118163CF520E030E040E251E46F85CC
:10069000788989899A890CD1DC01CB01BC01CD0113
:1006A0008AD0DC01CB01988F8F8B0FC080E991E05D
:1006B0009A8F898F898D9A8D0197F1F79A8F898FFB
:1006C0008F89988D0197988F8F8B8F89988D009740
:1006D00069F713C06B897C898D899E896CD0DC0198
:1006E000CB01988F8F8B8F89988D9C8F8B8F8B8D63
:1006F0009C8D0197F1F79C8F8B8FA3DDD7DCF6DC07
:1007000015DD34DD53DD72DD809160009091610074
:100710008732F2E09F0768F01092670080916000D6
:1007200090916100845F9140909363008093620098
:1007300088DD8091600090916100823C21E0920709
:1007400090F481E080936700809160009091610057
:1007500024EF31E0A901481B590BCA0190936300B3
:10076000809362006EDD8091600090916100823C18
:1007700051E0950780F08091600090916100873290
:10078000E2E09E0740F482E08093670010926300ED
:10079000109262004DDD909167008091660098177D
:1007A00029F08091670080936600AECFADCF2FD047
:1007B00008F481E0089557D088F09F5790F0B92F42
:1007C0009927B751A0F0D1F0660F771F881F991FA6
:1007D0001AF0BA95C9F712C0B13081F05ED0B1E01D
:1007E00008955BC0672F782F8827B85F39F0B93F2D
:1007F000CCF3869577956795B395D9F73EF49095A8
:100800008095709561957F4F8F4F9F4F0895990FF9
:100810000008550FAA0BE0E8FEEF16161706E807CA
:10082000F907C0F012161306E407F50798F0621BEB
:10083000730B840B950B39F40A2661F0232B242BC0
:10084000252B21F408950A2609F4A140A6958FEFDF
:10085000811D811D089557FD9058440F551F59F073
:100860005F3F71F04795880F97FB991F61F09F3F9D
:1008700079F087950895121613061406551FF2CFC6
:100880004695F1DF08C0161617061806991FF1CF16
:1008900086957105610508940895E894BB2766273D
:1008A0007727CB0197F90895B2DF08F48FEF089509
:1008B0000BD078C069D028F06ED018F0952309F0DD
:1008C0005AC05FC01124EACFC6DFA0F3959FD1F3D1
:1008D000950F50E0551F629FF001729FBB27F00DEE
:1008E000B11D639FAA27F00DB11DAA1F649F662743
:1008F000B00DA11D661F829F2227B00DA11D621F92
:10090000739FB00DA11D621F839FA00D611D221F4B
:10091000749F3327A00D611D231F849F600D211D2F
:10092000822F762F6A2F11249F5750408AF0E1F0D2
:1009300088234AF0EE0FFF1FBB1F661F771F881F1B
:1009400091505040A9F79E3F510570F014C0A6CFBA
:100950005F3FECF3983EDCF3869577956795B79506
:10096000F795E7959F5FC1F7FE2B880F911D969530
:10097000879597F9089597F99F6780E870E060E0A0
:1009800008959FEF80EC089500240A941616170628
:1009900018060906089500240A9412161306140670
:1009A00005060895092E0394000C11F4882352F0D3
:1009B000BB0F40F4BF2B11F460FF04C06F5F7F4F8B
:0A09C0008F4F9F4F0895F894FFCF6A
:00000001FF
